:020000000528D1
:10000800F3298B13831203138312031385018601CB
:100018008316FF30831603138500FF308600831292
:100028008B13063083120313A000A101A2018730AD
:1000380083168316031381008312C33083120313BC
:10004800D000D1018100A0308B00D201FF30D50152
:10005800D601DB00DC00D701D801DD00DE00D901C4
:10006800DA01DF00E000BB2883120313D400031079
:10007800520D553E8400831353088000840A5408A7
:100088008000D20A5208033A0319D2010310520D14
:100098008313553E84000008840A00040319452888
:1000A800801B452800088A00840300088200831208
:1000B80003134308C7004208023E0318C70A831304
:1000C8004718831784000008C4004308C700420883
:1000D800013E0318C70A83134718831784000008D2
:1000E800440603197828832883120313BF010130BB
:1000F800FF3ABF09013E0319BF0ABE00B5288312A3
:100108000313C701033044070318C70A4207C60090
:100118000318C70A4308C7078313471883174608F5
:1001280084000008C500C40A8313431883174208D3
:100138008400000844020318A228A5288312031388
:10014800C4014308C7004208023E0318C70A8313C4
:1001580047188317840044088000BF014508BE0083
:10016800B5288312031341088A004008820007302B
:10017800831203139F00B201B30101308400840786
:10018800553084078313B2308000840A033080001E
:100198005208013A031DD1284528023084008407FB
:1001A8005530840783138E308000840A063080001F
:1001B800831203135208023A031DE32845288312C9
:1001C8000313B70103110319EA28EB28ED29831259
:1001D80003133708003A0319F2280129F93083126A
:1001E8000313D3000030382845288312031321084D
:1001F8002206031D0029F828282983120313D40195
:100208000130D3005208840084075B3084078313CD
:10021800840A8017840353088000840A54088000E5
:100228001930D300013038284528831203132108D8
:100238002206031D28295208840084075B3084079E
:100248008313840A801F1829031103192C292D29C7
:10025800A22983120313C3012030C2000130C10058
:100268003A30C00000308A005B30820083120313EA
:100278003F08B9003E08B8000310B91F0314031C57
:1002880046294729A229831203133908BB003808D5
:100298007F39BA00BB010311BB1B582906303A0647
:1002A800031D582900303B0603195B297529831261
:1002B80003133908BB0038088039BA00BB013A0873
:1002C8003B04031968297129013083120313B20210
:1002D800031CB3038130B704742983120313371046
:1002E800A129831203133908BB0038087F39BA00E3
:1002F800BB010311BB1B862907303A06031D86295B
:1003080000303B0603198929A129831203133908F0
:10031800BB0038088039BA00BB013A083B0403190E
:1003280096299E2983120313B20A0319B30A82304D
:10033800B704A12983120313B710282983120313C2
:1003480037088039003A031DAA29D32983120313D9
:10035800B713D4010E30D3005208840084075B30F1
:1003680084078313840A8017840353088000840A4F
:1003780054088000C330D300013038284528831240
:10038800031321082206031DD2295208840084077A
:100398005B3084078313840A801FC229EC298312E7
:1003A800031337080139003A031DDB29E12901301D
:1003B80083120313B202031CB30337080239003A4D
:1003C800031DE729EC2983120313B20A0319B30AA0
:1003D800E6288312031335088A0034088200FF00D8
:1003E800030E8312031383120313CA00CA0E0A08EA
:1003F800CB000408CC000B1D1C2A5008810050308B
:10040800D107B4300318013EFF3A013ED0000B116A
:10041800FF30DC1B122ADB07031CDC07DE1B172A54
:10042800DD07031CDE07E01B1C2ADF07031CE007AF
:100438007C08CD007D08CE007E08CF004F08FE0066
:100448004E08FD004D08FC004C0884004B088A004B
:100458004A088300FF0E7F0E090083160313300835
:10046800B3002F08013E0318B30AB30183138400B5
:100478000008013EB2008313301883172F08840048
:10048800000832020318492A4C2A83160313B201C2
:100498003008B4002F08023E0318B40A8313341836
:1004A800831784000008320603195B2A622A013088
:1004B80083160313AC00AC09AC0A8E2A8316031307
:1004C8003008B4002F08013E0318B40A8313341807
:1004D80083178400B4010008033E0318B40A2F07E9
:1004E800B3000318B40A3008B40783133418831709
:1004F80033088400310880003008B4002F08013E1A
:100508000318B40A83133418831784003208800050
:10051800AC018E2A831603132E088A002D08820048
:1005280083120313AA01AB016908AC00AD01AE0147
:100538006A08AF006908831603138504831203133E
:100548006A08831603138604043083120313A90070
:100558006C08B1006B08B00068088A006708820060
:100568008312031330083104031DBB2AF72A013014
:1005780083160313A500A60108302602031CC52A0A
:10058800F72A8316031322082505003A031DCD2AEE
:10059800F12A8316031326082407A7002308250534
:1005A800003A031DD82ADB2A83160313A7178312E0
:1005B8000313310883160313B000831203133008A2
:1005C80083160313AF002708B1000230AE00F130E4
:1005D800AD0002308A003130820003108316031305
:1005E800A50DA60AC02A8316031321088A0020082D
:1005F8008200831203132C08003A031D042B2B2BB3
:10060800831203130508EC000508EB000508EC0449
:100618000508EB050508EC040508EB052B08EA00BE
:100628000508AB006A082B06E9002B08EC042B0828
:10063800EB056C086B06EA006A0869042C05003AA9
:10064800031D272B2B2B033083120313A9002F081C
:10065800003A031D302B572B831203130608EC00B6
:100668000608EB000608EC040608EB050608EC048F
:100678000608EB052E08EA000608AE006A082E06F2
:10068800E9002E08EC042E08EB056C086B06EA005E
:100698006A0869042F05003A031D532B572B0330B2
:1006A80083120313A9002908003A031D5C2BAC2B05
:1006B800FF3083120313A9072908003A0319652B91
:1006C800AC2B831203132A082B062C05E9006908B2
:1006D800003A031D702B882B831203132B082C055B
:1006E800AA00690883160313A200831203132A08B9
:1006F80083160313A300A4010330A1008830A000CF
:1007080002308A00B4308200831203132D082E06AB
:100718002F05E9006908003A031D932BAC2B8312BF
:1007280003132E082F05AD00690883160313A200D2
:10073800831203132D0883160313A3000830A400A3
:100748000330A100AC30A00002308A00B43082002F
:100758008312031368088A0067088200C030831276
:100768000313E900EA01EC012030EB000330E80054
:10077800C230E70002308A00943082000311031966
:10078800C62BC72BF42B033083120313E800D13098
:10079800E70002308A00FD30820083120313D30180
:1007A800D4015208840084075B3084078313840AC9
:1007B8008017840353088000840A54088000E830B6
:1007C800D3000330382845288312031352088400C5
:1007D80084075B3084078313840A801FE72BC22BAE
:1007E8008312031362088A006108820083160313C8
:1007F800D601D50104305502031C032C6D2C831639
:100808000313D3015508D2000310D20DD30D52089B
:10081800813E0318D30AD2000730D3075208D2000A
:100828001B2C8316031353088A00520882001524D0
:1008380083120317A90083160313D20A0319D30AD4
:10084800152483160313D30083120317290883166C
:100858000313D200D40103110319332C342C4C2C6C
:100868008316031353085102031C3E2C031D3E2C10
:1008780052085002031C412C422C4C2C83160313A3
:100888005208D002031CD1035308D102D40A2F2CDA
:10089800831603135408003A031D532C572C0130B8
:1008A80083160313D600D60803195B2C5C2C6B2C1B
:1008B800831603135408303ED70083134F18831749
:1008C8004E08840057088000CE0A0319CF0AD50ABB
:1008D800FE2B831603135008303ED70083134F189E
:1008E80083174E08840057088000CE0A0319CF0AE0
:1008F80083134F1883174E08840080014D088A001F
:100908004C0882008313831603134F1883174E086D
:1009180084000008003A031D922C982C83160313B8
:10092800CE0A0319CF0A862C031103199C2C9D2C7F
:10093800C32CA42C8316031351088A005008820084
:100948009E2483160313D20083134F1883174E086F
:1009580084005208800083134F1883174E088400C0
:100968000008003A0319B92CBA2CC32C83160313B8
:10097800CE0A0319CF0AD00A0319D10A982C831674
:1009880003134D088A004C088200043083160313B1
:100998006802031CD32C031DD32C003067020318F4
:1009A800D62CE72C013083120313D4000030D30077
:1009B8000000D30BDC2C0000003083160313E70281
:1009C800031CE803C92C0030831603136802031CB8
:1009D800F12C031DF12C043067020318F42C0A2DA6
:1009E80083160313680883120313D40083160313B2
:1009F800670883120313D3000310D40CD30C03101D
:100A0800D40CD30C0000D30B062D0000080071088D
:100A18007204031D102D1E2D83120313D401FA3006
:100A2800D3000000D30B152D00000130F102031C88
:100A3800F2030B2D08008312031385150800831297
:100A48000313851108008312031305158316031376
:100A5800670EF0398312031386040F3886050511D3
:100A680008002325710883160313E700E70E0F30EB
:100A7800E7052725710883160313E7002725831642
:100A88000313E8012830E700C92408001F2571086E
:100A980083160313E700E70E0F30E70527257108D3
:100AA80083160313E700272583160313E801323062
:100AB800E700C924080083160313061286120613DA
:100AC800861385110511F2010F30F1000B2523253E
:100AD800033083160313E7002725F2010530F100E0
:100AE8000B25033083160313E7002725831603130A
:100AF800E8016430E700C924033083160313E700D4
:100B08002725F2010530F1000B2502308316031367
:100B1800E700272583160313E8012830E700C924D6
:100B28002830F10035250830F10035250F30F10067
:100B380035250130F1003525F2010230F1000B2591
:100B48000630F1003525831603135C088A005B081C
:100B580082000C30F1003525831603135C088A00E7
:100B68005B088200831603135E080139F100F10E59
:100B7800F10DF10DC030F1058030F1045D083F3909
:100B8800F1043525831603135C088A005B0882008C
:100B9800831603135D080739F100F10DF10DF10D0E
:100BA800F830F1054030F104352583160313E001D0
:100BB80008306002031CE12DFE2D831603135F0825
:100BC800E2005E0860070318E20AE100F12D8316CF
:100BD800031362088A0061088200EB25F1004A25A8
:100BE80083160313E8015030E700C9248316031362
:100BF800E00ADC2D831603135C088A005B08820078
:100C0800063083160313DC000E30DB0005308A0043
:100C18005F308200831603134D088A004C08820057
:100C2800831603134E08DD004F08DE000630DC0093
:100C38002230DB0005308A00B630820083160313A9
:100C48004D088A004C088200063083160313DC0026
:100C58003230DB0005308A00AD3082008316031382
:100C68004D088A004C088200831603134E08DD00E5
:100C78005008DF004F08DE000630DC004830DB009B
:100C880005308A00CC30820083160313DD01DE01B3
:100C98000630DC005430DB0005308A00B6308200B4
:100CA800831603134D088A004C0882008316031329
:100CB8005D08F1004A25831603135C088A005B0867
:100CC80082008313831603134F1883174E0884007A
:100CD8000008003A031D712E882E83138316031310
:100CE8004F1883174E0884000008DD000630DC002A
:100CF8008230DB0006308A005A30820083160313E4
:100D0800CE0A0319CF0A652E831603134D088A00ED
:100D18004C088200063083160313CD009830CC00AF
:100D280006308A0004308200073083160313CE0091
:100D38000730D000C130CF000630CD00A830CC003D
:100D480006308A0038308200063083160313CD003F
:100D5800B230CC0006308A00283082008316031394
:100D6800C501C60103110319BA2EBB2E772F8312B2
:100D78000313330883160313C400831203133208C2
:100D880083160313C30083120313D301D40152083B
:100D9800840084075B3084078313840A80178403E4
:100DA80053088000840A54088000DE30D3000630DF
:100DB80038284528831203135208840084075B30BF
:100DC80084078313840A801FDD2E320883160313D9
:100DD8004306031DF52E83120313330883160313EA
:100DE8004406031DF82E3B2F83160313CF01B93099
:100DF800CE0083120313330883160313D100831222
:100E08000313320883160313D0000730CD001130C6
:100E1800CC0003308A00FA30820083160313CF0116
:100E2800B930CE000730D100C930D0000730CD002E
:100E38002230CC0004308A008630820083160313E7
:100E4800CE01CF010730CD002E30CC0006308A000D
:100E58001430820083160313CF01B930CE00073057
:100E6800CD003B30CC0006308A0065308200831606
:100E78000313CE010130CF000730CD004830CC003D
:100E880006308A0014308200831603134608C9000E
:100E98004508C8000310C90CC80C0310C90CC80CBD
:100EA80048080339C7000730C900BD304707031891
:100EB800C90AC800652F8316031349088A00480821
:100EC80082005F2783160313DD000730DC007130D2
:100ED800DB0006308A005A30820083160313C50AE5
:100EE8000319C60AB62E8316031338088A00370872
:100EF8008200643400340A34003410342734E8346F
:100F08000334643400340A3400340034CA349A3464
:100F18003B340034E134F534053480349634983465
:100F28000034403442340F340034A0348634013461
:100F380000341034273400340034E83403340034E7
:100F4800003464340034003400340A34003400348B
:100F58000034303431343234333434343534363484
:100F680037343834393441344234433444344534E2
:100F780046347C342F342D34073410340834083484
:0E0F88000434023402340134003420340034C6
:02400E00103F61
:00000001FF
